:020000040000FA
:020000000528D1
:08000800090083160313063002
:100010009F00003085003F308600C03087008B0194
:10002000811383120313432A7F0382075F345E34F4
:100030005D345C345B3482070034013402341034A4
:1000400001340634003410340234003409341034DE
:1000500010341034103410340134063400341034A9
:1000600006340434013410340034013402341034C2
:100070001034103410341034023400340934103485
:10008000003401340234103409340234083410349A
:10009000CB00CF010330D3006B083039CC004B08C4
:1000A0003039CD000310CD0C4D0CCC046C08303928
:1000B000CD004D0E4C041B20CE000339CF044E085A
:1000C0000C39CC00CC0DCC0DD30B6D286B080F393F
:1000D0004C04EB004F08EC000800CF0DCF0DCB0D0A
:1000E000CB0DEC0DEC0D4F28CB005539CF004B0854
:1000F000AA39CB000310CF0D4B0C4F04080003109E
:10010000CF00CF1E8628CF124F168B284F1ECF163A
:100110004F124F080800CF1D9028CF114F1595287A
:100120004F1DCF154F114F080800CF1C9A28CF1034
:100130004F149F284F1CCF144F104F0808004F0832
:10014000031408003F087F20BF00031C08003E087E
:100150007F20BE00031C08003D087F20BD00031C5B
:1001600008003C14080000084702031DBE28840A4A
:10017000840A0008403E8400000808000008670266
:10018000031DC928840A840A0008852383120313E7
:10019000080003010800CB0000084702031D080007
:1001A000840A840A0008403E84004B08800008004E
:1001B0006B1DDC28A030E128EB19E028A330E128F2
:1001C000A630840008006C18F528EC18F2286C1989
:1001D000F528EC19F2286C1AF528EC1AF2286B10A5
:1001E000EB1008006B14EB1008006B10EB14080008
:1001F0003D308400B320CB00A2283D308400B320E2
:10020000CC00A2203D308400B320CD00A2203D30A0
:100210008400B320CE00A2283D3084004C0880002A
:10022000840A4D088000840A4E08800008000330CC
:10023000D300CC016C1C21294B184C17CB18CC17C0
:100240002C29EC1C28294B1A4C17CB1ACC172C291B
:100250004B194C17CB19CC170310CC0CCC0CEC0C55
:10026000EC0CD30B1A2908004C08CF004E08CB0029
:1002700017214C08CE004D08CB0017214C08CD00AB
:100280004F08CB001721CB016D1C4B294C184B1488
:10029000CC18CB145629ED1852294E184B14CE18F1
:1002A000CB1456294D184B14CD18CB146D1D5D2958
:1002B0004C194B15CC19CB156829ED1964294E1929
:1002C0004B15CE19CB1568294D194B15CD19CB15EA
:1002D0006D1E6F294C1A4B16CC1ACB160800ED1A5E
:1002E00076294E1A4B16CE1ACB1608004D1A4B160D
:1002F000CD1ACB160800A2206E1CB5296E1D9029C0
:100300006E1E8629A03084006C08CB28EE1A8C293A
:10031000A33084006C08CB28A63084006C08CB285E
:10032000EE19A6296E1E97296C08EB000800EE1A3C
:10033000A329D8203D088000840A3E088000840A52
:100340003F08800008006C08ED0008006E1EAA2916
:10035000D820B029EE1AAE29D820B129D820B22948
:10036000840A840A6C0880000800EE18FE296E1DBD
:10037000DD296E1ECB290310EC0DEC0DEB1AEC14ED
:100380006B1A6C14EB12EC1BEB16EC136B126C1B60
:100390006B166C13E328EE1AD0296D084820E32869
:1003A000EB1AEC176B1A6C170310EC0C03186B1696
:1003B0000310EC0C0318EB16E328EE19F0296E1E5F
:1003C000E529F8204B08EC000800EE1AEB29F8208C
:1003D0004B084820E328F82017214C08EC00E328BC
:1003E0006E1EF529FD20D8200E29EE1AF929FD20D0
:1003F0000C29FD2034214B08EC00E3286E1D132A44
:100400006E1E072AA0308400B320EC000800EE1A0C
:100410000E2AA3308400B320EC000800A63084002C
:10042000B320EC000800EE19292A6E1E1A2A6B0868
:10043000EC000800EE1A262AD8200008BD00840A25
:100440000008BE00840A0008BF0008006D08EC0028
:1004500008006E1E312AD820840A840A0008EC00A5
:100460000800EE1A352AD8202D2AD8202E2A5B081B
:100470007420CC005C087420CD005D087420CE0090
:100480004C30840008003C3084003430FF00800190
:10049000840AFF0B472A1830C7001530C300FE300E
:1004A000FE000530FF007E08850014208400060948
:1004B00080007E1C3D09FE1C3E097E1D3F09FE1981
:1004C0006A2A3D308400B320EE006E095F186F0980
:1004D000DF186F097E1E6C098700DF1E982A7B21BA
:1004E000FF3087000314FE0DFF0B532A5F1E7D2A89
:1004F000BC184F2ABC147B214F2ABC105F1D862AD2
:100500003C194F2A3C1537220C214F2A3C11DF1C85
:100510008F2ADF19DC2C3722B320EF004F2A5F1C13
:100520004F2A5E087420EF0037226F08CB204F2A35
:100530000130F0000030F1000530F200C423702AD1
:02400E00723D01
:00000001FF
